:1000000001288316FF238F008B018C0164000730C9
:10001000810007309F000B3085008312203085005F
:1000200040309F001830A4001830A5002030A600F2
:100030002030A7007F30A800A9008030AB00AC00C2
:10004000AA0164300D2205182A148518AA14051572
:10005000051664300D22051C2A15851CAA15831669
:100060000830850083123F308500A001A3010430D1
:10007000A20008308B00851D4028640063003928E9
:10008000851D4028A00A85194228200C7F390D22A1
:10009000F73020070D22031085190314A30CA20BBF
:1000A00048286400A31F8428A2302007031C84284A
:1000B0008E30200703188428E03023060319872890
:1000C000F030230603199B28230E0739243E8400B1
:1000D0000830A200640085196A28200C2007FB3E26
:1000E0000D22031085190314A30CF73020070D22ED
:1000F000A20B7128851D8428AB17AC172308A31BFE
:1001000080008013ED21332868300D223328AA1790
:100110001230ED212408ED212508ED212608ED21DE
:100120002708ED212808ED212908ED212A08ED21D5
:100130003328AF139E28AF172C08AD00323085004E
:1001400083161A30850083120222AE1785186F2994
:1001500083168117831205146400AF1BC128413038
:100160009F0002221F151F19B3281E08B10064004A
:1001700051309F0002221F151F19BC281E08B00015
:10018000640059309F003C300D221F151F19C628EE
:100190001E083202031C003CB6001E08B2002530C7
:1001A0008500831681130D30850083120222051805
:1001B0006F29831681178312AE1385146400AF1B59
:1001C000F32849309F0002221F151F19E5281E0839
:1001D000B400640059309F0002221F151F19EE2839
:1001E0001E08B300640051309F003C300D221F15E3
:1001F0001F19F8281E083502031C003CB7001E0812
:10020000B5009F103F3085008316811308308500AC
:100210008312AF1B99280330360203189928033044
:1002200037020318992832083102031C992835082F
:100230003402031C9928AE01AF013008B10232022A
:10024000BB000310BB0CBA01BA0C8030B00024080C
:100250002507B002031C46293108B6002408B70060
:1002600088213808BA02031CBB033908BB02031CEF
:100270004629280AB7009B213108B6003008B7008C
:1002800088212B08BA002808B421AE003308B40234
:100290003502BB000310BB0CBA01BA0C8030B300AE
:1002A00026082707B302031C6F293408B600260866
:1002B000B70088213808BA02031CBB033908BB0207
:1002C000031C6F29290AB7009B213408B6003308A4
:1002D000B70088212C08BA002908B421AF002E08E5
:1002E000AB002F08AC0083160830850083123F3026
:1002F00085009F108030AD1B8629AE1F8229AB1769
:10030000AC178629AF172E08ED212F08ED213328D1
:10031000B801B901A101371C93293608B8070318A1
:10032000B90A2108B9070310B60DA10DB70CB7081B
:10033000031D8B290800BC01BD01BE01A101371CB2
:10034000AB293A08BC070318BD0A3B08BD070318D0
:10035000BE0A2108BE070310BA0DBB0DA10DB70CD4
:10036000B708031D9F290800B6000A30A100B70195
:100370000310B70D3608031808000310BC0DBD0D9F
:10038000BE0D36080318080038083D023908031C62
:10039000390A3E02031CD2293808BD023908031C61
:1003A000390ABE02A10BB929BA1BE529031CDF29B2
:1003B0000310BA0D370A3A060319B70AE5290314E0
:1003C000BA0D3A0A37060319B7030310B70C3608FB
:1003D00037023608031C370808008512A3000930CD
:1003E000A200F53020070D220314A30C031CFA29E8
:1003F0008516FC2985120000F43020070D22A20B7F
:10040000F4290800032A042A052A062A072A082AAA
:10041000092A0A2A0B2A0C2A0800A100F730A10792
:10042000F930A10703302105031D102AA10CA10CEE
:0C0430003F30A1056400A10B1A2A08004F
:0207FE00B03415
:084000000100010001000200B3
:02400E006C3F05
:00000001FF
